:100000000C9463000C948B000C948B000C948B006C
:100010000C948B000C948B000C948B000C94910727
:100020000C948B000C948B000C948B000C948B0024
:100030000C948B000C948B000C948B000C948B0014
:100040000C9447070C948B000C9415070C94EF0646
:100050000C948B000C948B000C948B000C948B00F4
:100060000C948B000C948B000000000023002600F1
:10007000290000000000240027002A0000000000E2
:10008000250028002B0004040404040404040202D4
:100090000202020203030303030301020408102007
:1000A0004080010204081020010204081020000012
:1000B0000008000201000003040700000000000027
:1000C00000005108C51911241FBECFEFD8E0DEBFD4
:1000D000CDBF23E0A0E7B1E001C01D92A839B2076F
:1000E000E1F711E0A0E0B1E0E6E5F2E402C005903E
:1000F0000D92A037B107D9F710E0C2E6D0E004C0F6
:100100002197FE010E94321CC136D107C9F70E9417
:1001100091090C941E210C9400000895AF92BF9297
:10012000CF92DF92EF92FF920F931F93CF93DF93C3
:100130006C017B018B01040F151FEB015E01AE18F2
:10014000BF08C017D10759F06991D601ED91FC9114
:100150000190F081E02DC6010995892B79F7C50141
:10016000DF91CF911F910F91FF90EF90DF90CF9093
:10017000BF90AF900895FC01538D448D252F30E042
:10018000842F90E0821B930B541710F0CF960895A4
:1001900001970895FC01918D828D981761F0A28DD1
:1001A000AE0FBF2FB11D5D968C91928D9F5F9F7397
:1001B000928F90E008958FEF9FEF0895FC01918D4D
:1001C000828D981731F0828DE80FF11D858D90E0BA
:1001D00008958FEF9FEF0895FC01918D228D892F57
:1001E00090E0805C9F4F821B91098F73992708953F
:1001F00083EC91E00E94EC0021E0892B09F420E0DF
:10020000822F0895FC01A48DA80FB92FB11DA35A08
:10021000BF4F2C91848D90E001968F739927848F26
:10022000A689B7892C93A089B1898C918370806449
:100230008C93938D848D981306C00288F389E02DEA
:1002400080818F7D80830895EF92FF920F931F939B
:10025000CF93DF93EC0181E0888F9B8D8C8D981379
:100260001AC0E889F989808185FF15C09FB7F89485
:10027000EE89FF896083E889F989808183708064D1
:1002800080839FBF81E090E0DF91CF911F910F911C
:10029000FF90EF900895F62E0B8D10E00F5F1F4F2B
:1002A0000F731127E02E8C8D8E110CC00FB607FC3A
:1002B000FACFE889F989808185FFF5CFCE010E94C8
:1002C0000201F1CFEB8DEC0FFD2FF11DE35AFF4F33
:1002D000F0829FB7F8940B8FEA89FB898081806256
:1002E000CFCFCF93DF93EC01888D8823B9F0AA8913
:1002F000BB89E889F9898C9185FD03C0808186FDE1
:100300000DC00FB607FCF7CF8C9185FFF2CF80812F
:1003100085FFEDCFCE010E940201E9CFDF91CF91A1
:100320000895833081F028F4813099F08230A9F06B
:1003300008958730A9F08830C9F08430B1F48091F5
:1003400080008F7D03C0809180008F778093800034
:10035000089584B58F7784BD089584B58F7DFBCFD4
:100360008091B0008F778093B00008958091B000A5
:100370008F7DF9CF1F93CF93DF93282F30E0F901C2
:10038000E255FF4F8491F901E656FF4FD491F901F0
:10039000EA57FF4FC491CC23A9F0162F81110E9478
:1003A0009101EC2FF0E0EE0FFF1FE458FF4FA591F5
:1003B000B4918FB7F894EC91111108C0D095DE2359
:1003C000DC938FBFDF91CF911F910895DE2BF8CF83
:1003D000CF93DF9390E0FC01E656FF4F24918A57BC
:1003E0009F4FFC0184918823D1F090E0880F991FE2
:1003F000FC01EE58FF4FA591B491FC01E458FF4F6A
:10040000C591D49161110EC09FB7F8948C91E22FE1
:10041000E0958E238C932881E223E8839FBFDF91B0
:10042000CF9108958FB7F894EC91E22BEC938FBFA6
:10043000F6CFCF93DF93EC0161E085E00E94E80105
:10044000209731F460E085E0DF91CF910C94BA0100
:10045000CF3FD10511F461E0F6CFE3EBF0E0E4919A
:10046000E33029F140F4E130B1F0E230D9F0C038A6
:10047000D1058CF7E7CFE73021F1E83051F1E430D6
:10048000B1F780918000806280938000D0938B00D0
:10049000C0938A0004C084B5806884BDC7BDDF9165
:1004A000CF91089584B5806284BDC8BDF8CF809196
:1004B0008000806880938000D0938900C09388007A
:1004C000EECF8091B00080688093B000C093B300FD
:1004D000E6CF8091B00080628093B000C093B400FA
:1004E000DECF8E3008F08E508770806480937C0061
:1004F00080917A00806480937A0080917A0086FDF2
:10050000FCCF809178009091790008953FB7F894DE
:100510008091750190917601A0917701B091780159
:1005200026B5A89B05C02F3F19F00196A11DB11D4E
:100530003FBFBA2FA92F982F8827BC01CD01620F8A
:10054000711D811D911D42E0660F771F881F991F45
:100550004A95D1F708958F929F92AF92BF92CF9212
:10056000DF92EF92FF926B017C010E9486024B01A9
:100570005C01C114D104E104F104B9F00E948602C7
:10058000681979098A099B09683E734081059105BC
:1005900080F321E0C21AD108E108F10888EE880E44
:1005A00083E0981EA11CB11CE4CFFF90EF90DF9078
:1005B000CF90BF90AF909F908F9008952FB7F894F1
:1005C0006091710170917201809173019091740139
:1005D0002FBF08958F929F92AF92BF92CF92DF92DA
:1005E000EF92FF920F931F936B017C010E94DE023A
:1005F00000916403109165032091660330916703B5
:100600004B015C01801A910AA20AB30A870130E00B
:1006100020E080169106A206B306F0F16093640311
:1006200070936503809366039093670360915B0307
:1006300070915C0380915D0390915E039B01281B88
:10064000390BA90137FF04C044275527421B530B20
:10065000EC2DF0E080915703909158038130910583
:1006600019F08430910521F581E0121613060CF47F
:1006700080E04E175F0714F0882331F18091610309
:100680008F5F8093610370935E0360935D0381E0ED
:10069000909161039D1508F480E01F910F91FF90E8
:1006A000EF90DF90CF90BF90AF909F908F90089584
:1006B0000297029730F4832F8095881F8827881F20
:1006C000D8CF4E175F07D4F210926103DCCFCF93DF
:1006D000DF93EC0188810E9471029A8389832B81C8
:1006E0003C81AC01421B530B9A0157FF03C031956B
:1006F000219531092230310514F09C838B838B8145
:100700009C81B0E0A0E02B853C85821B930BA10966
:10071000B109B7FF03C09C5FAF4FBF4F9A8789876E
:10072000BC0190E080E00E94301A20E030E044EB11
:1007300053E40E94911A20E030E040E85AE30E941E
:10074000911A6D837E838F839887DF91CF9108956F
:10075000CF93DF93C1E5D3E0188A8A819B810E9401
:100760006703EA81FB81818592859D878C870E9442
:10077000DE026B8B7C8B8D8B9E8BDF91CF910895EE
:100780002091550330915603232BA1F522E030E050
:1007900030935803209357039093600380935F0333
:1007A0000E94A8030E94DE026093680370936903AD
:1007B00080936A0390936B03E0915103F09152038D
:1007C00085E998E0A0E0B0E085839683A783B087B1
:1007D00080E694E5A0E0B0E0818B928BA38BB48B94
:1007E0008FEF9FEF968B858B81E090E0909356037F
:1007F000809355030895CF93DF9320915503309153
:100800005603232B81F5C1E0D0E0D0935803C09369
:1008100057039093600380935F030E94A8030E9494
:10082000DE02609368037093690380936A03909378
:100830006B03E0915103F091520385E998E0A0E049
:10084000B0E085839683A783B08780E694E5A0E037
:10085000B0E0818B928BA38BB48BD68BC58BD0935E
:100860005603C0935503DF91CF910895CF92DF9245
:10087000EF92FF920F931F93CF93DF93442331F1B5
:100880008C01D0E0C0E06B01770FEE08FF0861E05B
:1008900081E10E94BA01C701B6010E94AB0260E08B
:1008A00081E10E94BA0162E370E080E090E00E9482
:1008B000AB0221960C171D0751F7DF91CF911F91C5
:1008C0000F91FF90EF90DF90CF9008956E5C7F4F77
:1008D000072E000C880B990BDF91CF911F910F9180
:1008E000FF90EF90DF90CF900C94AB02EF92FF92CD
:1008F0000F931F93CF93DF937C0101EA11E0D0E0C7
:10090000C0E0F80161918F01C7018C0F9D1F0E940B
:10091000571B2196C232D105A1F782E290E0DF9108
:10092000CF911F910F91FF90EF90089580917E01DC
:1009300090917F010C9476040F931F93CF93DF93D4
:10094000C1EAD1E08C01015A1140C8018C0F9D1FF2
:100950000E944F1B899381E0C33CD807B1F782E224
:1009600090E0DF91CF911F910F910895FC0180815C
:100970009181009711F00C94EF1960E070E0CB01C9
:1009800008950F931F93CF93DF938C01EB01FC012C
:10099000808191810097E1F068817981611571050D
:1009A000A9F0428153812C813D814217530770F099
:1009B0000E94461E8C819D81F801958384831D824F
:1009C0001C82DF91CF911F910F9108950E94F71C17
:1009D00088819981F801918380838A819B819383A7
:1009E00082838C819D8195838483198218821B82E6
:1009F0001A82E5CFCF93DF93EC018881998100972C
:100A000011F00E94F71C198218821D821C821B8221
:100A10001A82DF91CF910895FC0180819181009726
:100A200011F00C94F71C08950F931F93CF93DF934D
:100A3000EC0188819981009759F02A813B81261722
:100A4000370730F081E0DF91CF911F910F9108952A
:100A50008B016F5F7F4F0E94801D009759F0998333
:100A600088831B830A832C813D81232B59F7FC014A
:100A70001082E8CF80E0E7CFEF92FF920F931F93B1
:100A8000CF93DF93EC01FB01E080F180E114F104EE
:100A900011F10481158101151105A9F08C819D8149
:100AA000080F191FB801CE010E941405882399F080
:100AB000288139818C819D81B701820F931F0E940B
:100AC000461E1D830C83CE01DF91CF911F910F91A4
:100AD000FF90EF900895CE010E94FA04F4CFEF92B8
:100AE000FF920F931F93CF93DF93EC017B018A0159
:100AF000BA010E94140581110BC0CE010E94FA04B4
:100B0000CE01DF91CF911F910F91FF90EF9008954B
:100B10001D830C83B701888199810E94461EF0CF06
:100B2000FC0111821082138212821582148250E01D
:100B300040E06EE671E00C946F05FB01019000202F
:100B4000E9F73197AF01461B570B0C946F05CF9314
:100B5000DF9300D0CDB7DEB7FC0111821082138283
:100B600012821582148269831A82BE016F5F7F4FE1
:100B70000E949D050F900F90DF91CF910895CF9324
:100B8000DF93EC01FB018617970749F060817181C3
:100B90006115710541F0448155810E946F05CE01B8
:100BA000DF91CF9108950E94FA04F9CFFF920F933D
:100BB0001F93CF93DF9300D0CDB7DEB786E0F82E3A
:100BC00083EC91E00E94EC00892B09F476C083EC61
:100BD00091E00E94CA00833251F08E3309F049C07F
:100BE0006EE671E088E393E00E949D05E9CF2091D5
:100BF00032033091330380913603909137032817E5
:100C00003907F4F6409134035091350320913003B5
:100C100030913103C90101969093310380933003E1
:100C2000F29EC001F39E900D112468E373E0840FDF
:100C3000951F0E94BF058091320390913303019666
:100C4000909333038093320380913003909131036A
:100C50002091360330913703281739070CF0B0CFB5
:100C60002F5F3F4F821B930B909331038093300390
:100C7000A7CF89831A8200913C0310913D030F5F37
:100C80001F4FB80188E393E00E941405882309F4FC
:100C900097CF209138033091390380913C03909194
:100CA0003D03BE016F5F7F4F820F931F0E94461E60
:100CB00010933D0300933C0383CF0F900F90DF917F
:100CC000CF911F910F91FF9008950E94F80081111C
:100CD0000C94D60508950F931F93CF93DF93CDB750
:100CE000DEB7A0970FB6F894DEBF0FBECDBF1F9240
:100CF00093E29F937F936F93282F082E000C330B62
:100D00003F938F9389E491E09F938F931F9280E2AA
:100D10008F938E010F5F1F4F1F930F930E944D1EE5
:100D2000F80101900020E9F73197AF01401B510B0A
:100D3000B80183EC91E00E948E000FB6F894DEBFFC
:100D40000FBECDBFA0960FB6F894DEBF0FBECDBFCD
:100D5000DF91CF911F910F9108950F931F93CF9320
:100D6000DF93CDB7DEB7A0970FB6F894DEBF0FBE06
:100D7000CDBF1F9293E29F937F936F93282F082EEE
:100D8000000C330B3F938F9381E591E09F938F93FA
:100D90001F9280E28F938E010F5F1F4F1F930F935F
:100DA0000E944D1EF80101900020E9F73197AF0134
:100DB000401B510BB80183EC91E00E948E000FB6EE
:100DC000F894DEBF0FBECDBFA0960FB6F894DEBF7D
:100DD0000FBECDBFDF91CF911F910F9108951F924C
:100DE0000F920FB60F9211242F933F934F935F935F
:100DF0006F937F938F939F93AF93BF93EF93FF93E3
:100E000083EC91E00E940201FF91EF91BF91AF91BD
:100E10009F918F917F916F915F914F913F912F9112
:100E20000F900FBE0F901F9018951F920F920FB644
:100E30000F9211242F938F939F93EF93FF93E09141
:100E4000D301F091D4018081E091D901F091DA01D0
:100E500082FD1BC090818091DC018F5F8F73209198
:100E6000DD01821741F0E091DC01F0E0ED53FE4F2F
:100E7000958F8093DC01FF91EF919F918F912F913E
:100E80000F900FBE0F901F9018958081F4CF1F9286
:100E90000F920FB60F9211242F933F938F939F932E
:100EA000AF93BF938091710190917201A0917301F2
:100EB000B09174013091700123E0230F2D3758F564
:100EC0000196A11DB11D2093700180937101909333
:100ED0007201A0937301B093740180917501909198
:100EE0007601A0917701B09178010196A11DB11D05
:100EF0008093750190937601A0937701B093780168
:100F0000BF91AF919F918F913F912F910F900FBE05
:100F10000F901F90189526E8230F0296A11DB11D72
:100F2000D2CF1F920F920FB60F9211242F933F939F
:100F30004F935F936F937F938F939F93AF93BF93E1
:100F4000CF93DF93EF93FF932091600230E0F9019C
:100F5000E255FF4F8491F901E656FF4FD491F90114
:100F6000EA57FF4FC491CC2379F081110E9491017F
:100F7000EC2FF0E0EE0FFF1FE859FF4FA591B49161
:100F8000EC91ED2381E009F480E02091630230913F
:100F900064022F5F3F4F309364022093630290916D
:100FA0002D03943618F095E09093610290916102C0
:100FB000933009F44CC0E0F4923011F19091620248
:100FC000992319F081116BC02D9AFF91EF91DF9158
:100FD000CF91BF91AF919F918F917F916F915F91D1
:100FE0004F913F912F910F900FBE0F901F9018952A
:100FF000943009F448C0953009F78111DFCF09C05A
:101000008111DCCF209163023091640224363105D6
:1010100028F41092640210926302D0CF10922D0334
:10102000E0912D0391E09E0F90932D03F0E020912D
:10103000630230916402EE0FFF1FE05AFD4F3683CA
:101040002583109264021092630293E019C08130EC
:1010500009F0B4CFE0912D0391E09E0F90932D0302
:10106000F0E02091630230916402EE0FFF1FE05A1E
:10107000FD4F36832583109264021092630294E040
:10108000909361029BCF882359F2209163023091A3
:1010900064022536310508F491CF95E0F1CF2D9803
:1010A00094CFEF92FF920F931F93CF93DF93109201
:1010B000C6011092C50188EE93E0A0E0B0E08093F5
:1010C000C7019093C801A093C901B093CA012BE353
:1010D00031E03093C4012093C30125EC30E030931C
:1010E000D0012093CF0124EC30E03093D201209343
:1010F000D10120EC30E03093D4012093D30121ECD6
:1011000030E03093D6012093D50122EC30E03093CB
:10111000D8012093D70126EC30E03093DA012093F8
:10112000D9011092DC011092DD011092DE011092C3
:10113000DF011092810310928203109283031092B8
:1011400084031092850310928603109287031092F5
:1011500088031092890310928A0310928B031092D5
:101160008C0310928D0310928E0310928F031092B5
:1011700090031092910321E030E030939303209389
:10118000920326E020937D0327E020937E0328E04E
:1011900020937F0329E0209380032FE020937003A6
:1011A00024ED33E030937C0320937B031092720391
:1011B00010927103109274031092730310927A03C9
:1011C00010927903109275031092760310927703B0
:1011D000109278032DE733E03093520320935103AC
:1011E00020E733E0309354032093530310925603C7
:1011F0001092550310925A031092590310925C03F7
:1012000010925B0310925E0310925D0310926003D4
:1012100010925F031092610320E230E03093630389
:101220002093620310926403109265031092660388
:1012300010926703109268031092690310926A0378
:1012400010926B0310926D0310926C0310926F0357
:1012500010926E0324E020936002109262022AE052
:1012600020933E0310923F038093400390934103E9
:10127000A0934203B093430310924403109245039A
:1012800010924603109247031092480310924903AC
:1012900010924A0310924B0384E690E0A0E0B0E085
:1012A00080934C0390934D03A0934E03B0934F0350
:1012B0001092500388E393E00E94900510922F0350
:1012C00010922E03109231031092300310923303C8
:1012D0001092320384E190E09093370380933603B9
:1012E00080E890E00E945B1CEC0125E130E029934E
:1012F00039938E017C0120E8E20EF11CC8010E94A6
:1013000090050A5F1F4FE016F106C1F7D093350331
:10131000C0933403DF91CF911F910F91FF90EF9015
:101320000895CF93DF93CDB7DEB7C556D1090FB679
:10133000F894DEBF0FBECDBF789484B5826084BDC3
:1013400084B5816084BD85B5826085BD85B58160C9
:1013500085BD80916E00816080936E001092810047
:101360008091810082608093810080918100816002
:1013700080938100809180008160809380008091C3
:10138000B10084608093B1008091B000816080934F
:10139000B00080917A00846080937A0080917A0016
:1013A000826080937A0080917A00816080937A00D5
:1013B00080917A00806880937A001092C100E09159
:1013C000D301F091D40182E08083E091CF01F091CC
:1013D000D0011082E091D101F091D2018FEC808395
:1013E0001092DB01E091D701F091D80186E0808373
:1013F000E091D501F091D601808180618083E091F8
:10140000D501F091D601808188608083E091D5017B
:10141000F091D601808180688083E091D501F091C0
:10142000D60180818F7D808383EC91E00E94EC0067
:10143000892B29F083EC91E00E94CA00F5CF61E08E
:1014400081E10E94E80161E085E00E94E80161E03D
:1014500082E00E94E80161E08AE00E94E80101E880
:10146000E02E03E0F02E0DE713E061E0D8018D914E
:101470008D010E94E801F801319760E080810E94AF
:10148000BA01E016F10689F7EDE7F3E06496FFAFE5
:10149000EEAF649760E06496AEADBFAD64978D919A
:1014A0006496BFAFAEAF64970E94BA016496EEAD8A
:1014B000FFAD64970E171F0769F760E08091700316
:1014C0000E94E801809170030E9471029093720360
:1014D000809371039093740380937303B0E0A0E052
:1014E00020917B0330917C03821B930BA109B109EE
:1014F000B7FF03C09C5FAF4FBF4F90937A038093B9
:101500007903BC0190E080E00E94301A20E030E0D6
:1015100044EB53E40E94911A20E030E040E85AE3A3
:101520000E94911A609375037093760380937703FA
:101530009093780380915303909154030E94670322
:10154000E0915303F09154038185928590935E035B
:1015500080935D038091C1019091C20190936303D8
:1015600080936203893C910530F084E690E090938B
:1015700063038093620361E080913E030E94E8016F
:1015800060E080913E030E94BA0188EE93E0A0E003
:10159000B0E08093400390934103A0934203B09343
:1015A00043030E94DE0260934803709349038093D3
:1015B0004A0390934B0381E08093500384E690E0CC
:1015C000A0E0B0E080934C0390934D03A0934E03B2
:1015D000B0934F036EE671E088E393E00E949D05AF
:1015E00010927F0110927E0110927D0182E290E0C4
:1015F00090937C0180937B018EE190E090937A013F
:101600008093790110E000E0FF24F394C8010E9468
:101610009C048091A1019091A2018336910531F43F
:1016200010937F0100937E01F0927D010E5D1F4FAC
:101630000C3FF3E01F0751F700917E0110917F01ED
:1016400080917D01882309F4DDC1C8010E949C04BA
:101650001092A2011092A101C8010E94760420916B
:101660007B0130917C0180917E0190917F01820FFE
:10167000931F90937F0180937E0160917901709117
:101680007A01269FA001279F500D369F500D1124EF
:101690008417950724F010927F0110927E0183E653
:1016A00090E09093A2018093A10180917E0190919E
:1016B0007F010E9476048091BF019091C001845601
:1016C00091098538934030F084ED93E09093C00108
:1016D0008093BF018091C1019091C201893C910525
:1016E00030F084E690E09093C2018093C101809134
:1016F000AB01882321F061E082E00E94BA0164E638
:1017000070E080E090E00E94AB028091A701909190
:10171000A801019709F0D4C18091A9019091AA0173
:101720000E941902A091BD01A53608F0A4E6A0937D
:101730003F03209140033091410340914203509177
:101740004303B0E00E94651B24E630E040E050E037
:101750000E94101C2093440330934503409346039A
:10176000509347032115310541055105A9F080919A
:101770004C0390914D03A0914E03B0914F03281755
:1017800039074A075B0740F480934403909345036D
:10179000A0934603B09347032091BF013091C0014D
:1017A00030937C0320937B038091730390917403A7
:1017B000B0E0A0E0821B930BA109B109B7FF03C001
:1017C0009C5FAF4FBF4F90937A0380937903BC0126
:1017D00090E080E00E94301A20E030E044EB53E4D7
:1017E0000E94911A20E030E040E85AE30E94911AEA
:1017F00060937503709376038093770390937803D7
:101800008091C1019091C201893C910520F490938F
:10181000630380936203F89482E08093B000809326
:10182000B10094E69093B3001092B20080937000E0
:1018300078948093610210922D038091600260E0A1
:101840000E94E8014091B60166E970E081E090E015
:101850000E94360415E9412E18E0512E612C712C9E
:1018600080911F0190912001A0912101B09122014E
:10187000A6968CAF9DAFAEAFBFAFA6979091230158
:101880006B969FAF6B97A09124016C96AFAF6C974E
:10189000B09125016D96BFAF6D97E09126016E96D0
:1018A000EFAF6E976F969FAF6F97A096AFAFA09771
:1018B000A196BFAFA197A296EFAFA29780913203F6
:1018C00090913303181619060CF063C1CE01845BA6
:1018D0009F4F0E949005CE018A5B9F4F0E9490050A
:1018E0008091320390913303009709F448C18E012F
:1018F0000F5F1F4F181619060CF4E5C0CE018E9627
:101900000E949005BE01625D7F4FCE01845B9F4FB8
:101910000E94C104CE018E960E940C056296CEAC48
:10192000DFAC6297AA24A394B12CC114D10421F096
:101930005601CC24C394D12CC8010E949005629614
:10194000EEACFFAC6297CE14DF0408F5AE14BF0412
:1019500008F475012E96EEADFFAD2E97EE0DFF1D2E
:10196000B08010822E966EAD7FAD2E976C0D7D1DD2
:10197000C8016115710509F4F0C00E949D052E96FD
:101980008EAD9FAD2E97E80EF91ED701BC92B8011F
:10199000CE018A5B9F4F0E94C104C8010E940C05C2
:1019A00062968EAD9FAD6297892B09F4E8C02E96A2
:1019B000EEADFFAD2E97309709F4E1C0E081E2541F
:1019C000E83108F0DCC00E2E000CFF0BE651F34F9F
:1019D0000C94321C4D0F0E0F3D0FDE10A710191284
:1019E000B00DBF0D880F1012270F0B11C111F50E8E
:1019F000EC12BF0D6E11990FCF0F6D12E70E23126F
:101A0000DF0F941083E690E09093A2018093A101F0
:101A100081E290E09093A4018093A30181E090E0A3
:101A20009093A6018093A5011092A8011092A7019E
:101A30001092AA011092A9018093AB0122E030E03C
:101A40003093AD012093AC0122E130E03093AF013F
:101A50002093AE0120E430E03093B1012093B00137
:101A600020E830E03093B3012093B2012EEF30E054
:101A70003093B5012093B4018093B6011092B80160
:101A80001092B7018DE290E09093BA018093B90172
:101A90008CEB92E09093BC018093BB011092BE014D
:101AA0001092BD0184ED93E09093C0018093BF013B
:101AB00084E690E09093C2018093C101C801F9CD02
:101AC00090E080E02DCE20912E0330912F0346E050
:101AD000429FC001439F900D112460913403709187
:101AE0003503680F791F1A8219821C821B821E829D
:101AF0001D82C8010E94BF0580912E0390912F0383
:101B0000019690932F0380932E03209132033091FE
:101B10003303215031093093330320933203209152
:101B20003603309137032817390744F42F5F3F4FAE
:101B3000821B930B90932F0380932E031FA61EA648
:101B400019AA18AA1BAA1AAAB801CE018E960E9439
:101B5000C104C8010E940C05D5CE0E94FA040FCF23
:101B60006CE071E0C8010E94461E64E670E080E00F
:101B700090E00E94AB02B80188E40E946B06CE019F
:101B80008A5B9F4F0E940C05CE01845B9F4F0E9491
:101B90000C0585E692E090939901809398018091DD
:101BA0002D03282E312C30929B0120929A01809196
:101BB0006102853009F0D9C0809167029091680276
:101BC000885891098D35910508F05CC580912D03E9
:101BD000843009F029C58091690290916A0280974A
:101BE000479708F021C580916B0290916C0209978C
:101BF000099708F019C510929701109296018FEF7E
:101C00009FEFDC018093920190939301A093940144
:101C1000B093950181E090E090938F0180938E01C5
:101C20000E94DE024B015C01809192019091930130
:101C3000A0919401B09195018F3FFFEF9F07AF07EF
:101C4000BF0709F0C5C580918A0190918B01A091D1
:101C50008C01B0918D018093920190939301A09398
:101C60009401B093950181E080938901C0908A012D
:101C7000D0908B01E0908C01F0908D0180918401D7
:101C800081112DC02DE3C21622ECD2062AE9E2060C
:101C900026EAF20649F047E6C41648E9D4064AE9BE
:101CA000E40646EAF406D9F48091A7019091A801D0
:101CB000019711F00C94FF188091B7019091B80131
:101CC000892B11F00C9484194091B60164E670E000
:101CD00081E090E00E94360481E08093840187E6F1
:101CE000C81688E9D8068AE9E80686EAF80609F4FB
:101CF000CCC60CF088C5ADEFCA16A2E0DA06AAE998
:101D0000EA06A6EAFA0609F4BBC5BDEDCB16B2E2B7
:101D1000DB06BAE9EB06B6EAFB0611F40C942019CF
:101D20008091A7019091A8010197D1F48091B7010A
:101D30009091B801892BA1F480918101882381F0D1
:101D400064E670E080E090E00E94AB024091B60152
:101D500064E670E082E090E00E9436041092810117
:101D600082E08093610210922D03809150038823BA
:101D700009F429C70E94DE0200914803109149032B
:101D800020914A0330914B036B017C01C01AD10AA8
:101D9000E20AF30A009140031091410320914203AB
:101DA00030914303C016D106E206F30640F060937B
:101DB00048037093490380934A0390934B03209107
:101DC0003E0330913F033111E0C660E0F9C668E0A0
:101DD00071E0C8010E94461E64E670E080E090E079
:101DE0000E94AB02B80186E5C8CE4091B60168EC0E
:101DF00070E081E090E00E94360481E090E09093F2
:101E0000B8018093B7011092A6011092A5018091AC
:101E1000BB019091BC010E94FB03B1CE4091B60181
:101E200068EC70E081E090E00E94360482E090E08F
:101E30009093B8018093B7011092A6011092A5016A
:101E40008091B9019091BA010E94C00398CE81E0BF
:101E500090E09093A8018093A7010E94960480913E
:101E6000A9019091AA010E9419026091A9017091A3
:101E7000AA018CE40E94AD0682CE1092A8011092B5
:101E8000A7010E94960490E080E00E9419026091F0
:101E9000A9017091AA0184E4EDCFCE018A5B9F4F26
:101EA0000E94B60497FD2EC06F3F71058105910514
:101EB00009F05CF57093AA016093A9018091A701D4
:101EC0009091A801019719F4CB010E9419020E9478
:101ED00096048091AA018F938091A9018F9389E53F
:101EE00091E09F938F931F930F930E947D1EB801E3
:101EF00082E40E946B060F900F900F900F900F904E
:101F00000F903DCE70E060E0D5CF6FEF70E0D2CFA4
:101F10008091AA018F938091A9018F9389E591E027
:101F20009F938F931F930F930E947D1EB8018AE4A5
:101F3000E0CF8091BC018F938091BB018F93809102
:101F4000BA018F938091B9018F938091BE018F93D5
:101F50008091BD018F938091A6018F938091A501FF
:101F60008F938091A8018F938091A7018F93809187
:101F7000B8018F938091B7018F938CE591E09F9387
:101F80008F931F930F930E947D1EB80183E50E94DB
:101F90006B060FB6F894DEBF0FBECDBFF0CDCE01FD
:101FA0008A5B9F4F0E94B604672B29F41092B601FA
:101FB0000E949604E4CD81E08093B601F9CFECEA6B
:101FC000CE2EE1E0DE2EF2E0EF2EF12C2C968EAD3F
:101FD0009FAD2C97E816F90638F42896EEADFFADC4
:101FE0002897309709F091C010928001E0E8F1E065
:101FF0006081C8010E94A705C70101972C962EADEC
:102000003FAD2C978217930738F42896EEADFFADBD
:102010002897309709F07CC010928001E0E8F1E049
:102020006081CE018E960E94A705C70102972C966B
:102030002EAD3FAD2C978217930738F42896EEAD5E
:10204000FFAD2897309709F066C010928001E0E854
:10205000F1E06081CE01CA960E94A7051DAA1CAAC4
:102060001FAA1EAA19AE18AEBE01665C7F4FCE0134
:10207000C4960E94BF05BE01625D7F4FCE01C4962B
:102080000E943C05B8010E943C0522961FAE1EAE80
:10209000229724961FAE1EAE249726961FAE1EAE24
:1020A0002697BC01CE01805C9F4F0E94BF05CE01E8
:1020B000C4960E940C05CE01CA960E940C05CE0162
:1020C0008E960E940C05C8010E940C05CE01805C12
:1020D0009F4F0E94B60497FD21C06F3F7105810597
:1020E000910509F0F4F4D6016D937D936D01CE0155
:1020F000805C9F4F0E940C05B3E0EB0EF11CE1E108
:10210000EE16F10409F062CF53CFEE0DFF1D70CF34
:10211000E80FF91F85CFE80FF91F9BCF70E060E053
:10212000E2CF6FEF70E0DFCFCE018A5B9F4F0E945E
:10213000B604672B39F41092AB0160E082E00E9494
:10214000BA0136CF81E08093AB0161E0F7CF6CE25A
:1021500071E080E090E00E94AB0280E793E00E9493
:1021600067038091790390917A039C012150310992
:102170002F36334000F59093BA018093B901109245
:10218000B8011092B70181E090E09093A60180938E
:10219000A5010E9496046091B9017091BA0186E48C
:1021A0000E94AD064091B60164E670E082E090E0E6
:1021B0000E943604E4CC8DE290E0DDCF6CE271E069
:1021C00080E090E00E94AB0280E793E00E9467030A
:1021D0008091790390917A039C01215031092F3627
:1021E0003340B0F49093BC018093BB011092B801CE
:1021F0001092B70182E090E09093A6018093A50130
:102200000E9496046091BB017091BC0185E4C8CF27
:102210008CEB92E0E7CFCE018A5B9F4F0E94B60421
:10222000DB0121E230E00E94381C6B017C01C1140B
:10223000D104E104F10409F4A2CC85E090E090938C
:10224000B8018093B7011092A6011092A501809168
:10225000550390915603892B09F091CC81E090E0D1
:10226000F7FE02C082E090E09093580380935703FA
:102270001092600310925F030E94A8030E94DE0286
:10228000609368037093690380936A0390936B0370
:10229000E0915103F0915203458256826782708625
:1022A000D701C601F7FE07C088279927DC018C19E2
:1022B0009D09AE09BF09818B928BA38BB48B81E002
:1022C00090E0F7FE02C08FEF9FEF968B858B81E049
:1022D00090E0909356038093550351CC4091B60102
:1022E00068EC70E081E090E00E9436048091550334
:1022F00090915603892BF1F504E010E010935803F8
:10230000009357030E94A8030E94DE0260936803B3
:102310007093690380936A0390936B03E091510378
:10232000F0915203458256826782708680915303F2
:10233000909154030E946703E0915303F09154037A
:102340008185928590935A0380935903E0915103BC
:10235000F091520380E694E5A0E0B0E0818B928B8F
:10236000A38BB48B81E090E0968B858B1093560302
:102370000093550384E090E09093B8018093B701F7
:10238000FECB4091B60168EC70E081E090E00E94E5
:1023900036048091550390915603892BF1F503E0A3
:1023A00010E010935803009357030E94A8030E9463
:1023B000DE02609368037093690380936A039093CD
:1023C0006B03E0915103F09152034582568267827C
:1023D000708680915303909154030E946703E091AB
:1023E0005303F09154038185928590935A0380930F
:1023F0005903E0915103F091520380E694E5A0E087
:10240000B0E0818B928BA38BB48B8FEF9FEF968B79
:10241000858B109356030093550383E090E0ACCF77
:1024200010928E0310928F031092900310929103DA
:10243000A6CB80E793E00E946703609179037091D7
:102440007A0387E417CDCE018A5B9F4F0E94B604C2
:10245000DB0177FF02C0B0E0A0E0A536B10514F0C3
:10246000A4E6B0E0B093BE01A093BD01A0933F03EA
:102470002091400330914103409142035091430326
:102480000E943F1C24E630E040E050E00E94101C17
:1024900020934403309345034093460350934703EE
:1024A000211531054105510509F482CD80914C0378
:1024B00090914D03A0914E03B0914F032817390717
:1024C0004A075B0708F074CD80934403909345035B
:1024D000A0934603B09347036BCD2C968EAD9FAD72
:1024E0002C97892B09F46CC0CE018A5B9F4F0E9408
:1024F000B60497FD6BC06115A4E07A0781059105CC
:102500000CF067C00091BF011091C001061B170BB2
:102510007093C0016093BF0170937C0360937B0351
:102520008091730390917403B0E0A0E0AB01770F4A
:10253000660B770B841B950BA60BB70BB7FF03C07D
:102540009C5FAF4FBF4F90937A0380937903BC0198
:1025500090E080E00E94301A20E030E044EB53E449
:102560000E94911A20E030E040E85AE30E94911A5C
:102570006093750370937603809377039093780349
:102580008091BB019091BC01800F911F9C5F20E066
:1025900034E0B9010E94FC1B9093BC018093BB0105
:1025A0008091B9019091BA01800F911F9C5FB90190
:1025B0000E94FC1B9093BA018093B9010E9496047B
:1025C0006091BF017091C00185E554CC70E060E07E
:1025D00099CF6FEF73E096CF2C968EAD9FAD2C9771
:1025E000892BB1F0CE018A5B9F4F0E94B60497FD04
:1025F00015C0693C7105810591059CF47093C20179
:102600006093C10170936303609362030E94960418
:102610006091C1017091C20180E52CCC70E060E056
:10262000EDCF68EC70E0EACF80912D03843450F157
:102630008091690290916A02825491098E9710F5F7
:1026400030E020E080E090E0DC01F901E559FD4F49
:1026500040815181495051094930510598F4F9019F
:10266000E359FD4F40815181465151094131510596
:1026700008F486C0408151814650510947305105C8
:1026800008F490C0B6E02B1631040CF469CB00E6D8
:1026900012E0E3E0F0E06696FFAFEEAF669755EC30
:1026A000C52E5DE9D52E5CE1E52E51E8F52E669646
:1026B0008EAD9FAD6697821593050CF078C0D8015A
:1026C0001B966D917C911C971796AD90BC9090E0F5
:1026D00080E00E94301A6A966CAF7DAF8EAF9FAFDC
:1026E0006A97B50190E080E00E94301A4B015C01CE
:1026F0002DEC3CEC4CE45FE30E94911A9B01AC0191
:102700006A966CAD7DAD8EAD9FAD6A970E942B1A17
:10271000F0E0E0E087FD18C02DEC3CEC4CE45FE31A
:102720006A966CAD7DAD8EAD9FAD6A970E94911A91
:102730009B01AC01C501B4010E942B1AE2E0F0E05C
:1027400087FD02C0E1E0F0E0A701960163E971E0D6
:1027500080E091E00E94EC1B6F01FF0FEE08FF0884
:10276000C626D726E826F9266696EEADFFAD669713
:1027700031966696FFAFEEAF66970E5F1F4F97CF0D
:10278000880F991FAA1FBB1F81602C5F3F4F203805
:10279000310509F05ACF20E230E0309397012093C1
:1027A000960130CA880F991FAA1FBB1FEECFC09297
:1027B0009201D0929301E0929401F092950180E20F
:1027C00090E090939701809396018FEF9FEF24CA3A
:1027D00080938A0190938B01A0938C01B0938D011B
:1027E0001092890180E991E09093010180930001AA
:1027F0008092850190928601A0928701B092880113
:102800001092840133CAE7E5CE16E8EADE06EAE96B
:10281000EE06E6EAFE0609F498C0FDE3CF16F2ECF8
:10282000DF06FAE9EF06F6EAFF0609F42EC12DE508
:10283000C21622EAD2062AE9E20626EAF20609F0E0
:102840006FCA4091B60164E670E081E090E00E94BA
:1028500036048091A5019091A6018130910509F07F
:10286000F9C09093B8018093B7011092A60110921D
:10287000A5018091BB019091BC010E94FB0350CA4D
:102880008091B7019091B801892B09F049CA409114
:10289000B60164E670E081E090E00E943604809129
:1028A000A7019091A801892BB1F481E090E0909369
:1028B000A8018093A7018FEF9FEF909383018093EE
:1028C00082018091A9019091AA010E94190281E0E0
:1028D0008093A00125CA1092A8011092A70190E050
:1028E00080E0F3CF0E94DE02C0908501D090860187
:1028F000E0908701F0908801AB01BC014C195D09A3
:102900006E097F098091000190910101B0E0A0E083
:10291000481759076A077B0708F0A6C401CA8091C7
:10292000AB018111FDC911E01093AB0161E082E0C0
:102930000E94BA014091B60164E670E082E090E046
:102940000E9436041093A001EBC98091A7019091D9
:10295000A801019709F004CA8091B7019091B801CC
:10296000892B09F0E3C910918901111142C00E941D
:10297000DE026093850170938601809387019093B6
:102980008801111153C04091B60164E670E081E006
:1029900090E00E943604009182011091830110168C
:1029A000110614F001E010E00150110910938301A9
:1029B000009382010115110509F47DC4000F111F58
:1029C000F801EF55FE4F838594859093AA0180937B
:1029D000A9010E9419028091A9019091AA018F3F3B
:1029E000910519F0019709F072CF81E08093810180
:1029F0006ECF0E94DE02C0908501D0908601E090EB
:102A00008701F0908801AB01BC014C195D096E098A
:102A10007F098091000190910101B0E0A0E048178A
:102A200059076A077B0708F0A2CF7AC98091AB01EA
:102A3000882309F475C91092AB0160E082E00E941E
:102A4000BA014091B60164E670E082E090E00E9435
:102A500036043DCF8230910579F49093B80180938C
:102A6000B7011092A6011092A5018091B901909131
:102A7000BA010E94C00354C910928E0310928F03B2
:102A800010929003109291034BC98091A7019091ED
:102A9000A801019709F064C98091B7019091B8012C
:102AA000892B09F043C9109189011123D1F080913C
:102AB000850190918601A0918701B0918801B501AF
:102AC000A401481B590B6A0B7B0B8091000190916C
:102AD0000101B0E0A0E0481759076A077B0708F436
:102AE00025C98092850190928601A0928701B092BB
:102AF00088013091A9012091AA01832F922F4DE3E3
:102B0000C41642ECD4064AE9E40646EAF40699F50E
:102B10008F3F910514F08EEF90E001969093AA01FB
:102B20008093A9018091A9019091AA010E941902A4
:102B30008091A9019091AA018F3F910511F0019711
:102B400019F481E08093810181E08093A001112339
:102B500009F4E6C880910001909101018333910549
:102B600008F4DEC844978233910560F09093010128
:102B700080930001D5C88230910514F482E090E082
:102B80000197CCCF82E390E0F1CFC0904803D09082
:102B90004903E0904A03F0904B036C197D098E09BC
:102BA0009F09C0904403D0904503E0904603F09005
:102BB00047036C157D058E059F0508F006C961E089
:102BC000822F0E94BA018091550390915603892B60
:102BD00009F4FDC00E94DE020091680310916903B0
:102BE00020916A0330916B03601B710B820B930B76
:102BF0006135734C8105910578F0E0915103F091B6
:102C00005203118A128A138A148A86E090E0909304
:102C1000560380935503DBC0809153039091540376
:102C20000E946703E0915303F091540381859285DC
:102C300090935C0380935B0320915503309156037E
:102C40002130310509F01FC220915F0330916003EC
:102C5000409157035091580311E02115310509F4B3
:102C6000E1C14130510541F48217930750F4803798
:102C7000934038F410E005C02817390710F4892B69
:102C8000C9F76F966FAD6F97A0967FADA097A1968D
:102C90008FADA197A2969FADA2970E94EA02112341
:102CA00009F48FC0E0915103F0915203118A128A06
:102CB000138A148A6CE271E080E090E00E94AB021B
:102CC00080915303909154030E946703E091530352
:102CD000F09154030185128510935C0300935B030C
:102CE000809157039091580360915F037091600346
:102CF000019709F060C0FB01E01BF10B8F0117FD8C
:102D0000BFC1C12CD12CE12C3FE3F32E02301105C1
:102D100034F0C12CD12C20E8E22E2FE3F22E60916A
:102D200062037091630390E080E00E94301AA70173
:102D300096010E94911A0E94B61B6B017C01B8019A
:102D4000110F880B990B0E94321A2AE939E945E3E1
:102D500051E40E94911A0E94B61BC60ED71EE81EAF
:102D6000F91E1C141D041E041F040CF089C10E94CE
:102D7000A8030E94DE026093680370936903809346
:102D80006A0390936B03E0915103F09152034582E3
:102D90005682678270868091570390915803C18A4A
:102DA000D28AE38AF48A8130910541F4968B858B2F
:102DB00082E090E02CCF061B170BA1CF8FEF9FEF87
:102DC000F5CFE0915103F0915203811155C18091EB
:102DD0008E0390918F03A0919003B0919103892B62
:102DE0008A2B8B2B09F48DC08091820390918303F1
:102DF000A0918403B0918503892B8A2B8B2B09F436
:102E000080C00E9486020091860310918703209162
:102E10008803309189036B017C01C01AD10AE20A50
:102E2000F30A00918203109183032091840330916F
:102E30008503C016D106E206F30608F462C060936B
:102E4000860370938703809388039093890380910E
:102E500081032091920330919303820F932F911D50
:102E6000049664E070E00E94FC1B809381038C0157
:102E70001127000F111F000F111F095D1E4F9DE745
:102E8000E92E93E0F92ED8016D918D01F701819122
:102E90007F010E94BA0164968EAD9FAD64978E1536
:102EA0009F0589F78091920390919303092E000C5E
:102EB000AA0BBB0B40918A0350918B0360918C034A
:102EC00070918D03840F951FA61FB71F80938A03EF
:102ED00090938B03A0938C03B0938D0380918E030A
:102EE00090918F03A0919003B09191030197A10954
:102EF000B10980938E0390938F03A0939003B093B6
:102F0000910380915503909156030597029708F01D
:102F10004DC064EF71E080E090E00E94AB0280E77A
:102F200093E00E9467038091B7019091B8018330CC
:102F3000910509F448C108F005C18130910509F4F3
:102F40000CC1029709F415C1809155039091560365
:102F5000069731F483E090E09093A6018093A50159
:102F60001092B8011092B7010091510310915203D1
:102F70007801E4E0EE0EF11C60E0D8018D918D0146
:102F80000E94BA01E016F106B9F7109256031092AA
:102F900055031092610381E08093A0014091B60136
:102FA00064E670E082E090E00E9436048091A00127
:102FB000813071F50E94DE0200919C0110919D010B
:102FC00020919E0130919F016B017C01C01AD10AB2
:102FD000E20AF30AB9E8CB16B3E1DB06E104F10437
:102FE00028F4601771078207930790F460939C019F
:102FF00070939D0180939E0190939F0183E690E0E2
:103000009093A2018093A1010E9496041092A001C6
:103010000E94F800882311F40C945E0C0E94D605DF
:103020000C945E0C4130510529F48037934020F414
:1030300010E002C0892BE1F76F966FAD6F97A096F5
:103040007FADA097A1968FADA197A2969FADA297B5
:103050000E94EA02E0915103F091520341895289A2
:103060006389748914161506160617062CF41111B7
:1030700003C0882309F4ABCE118A128A138A148AFA
:1030800085E090E0C4CD22303105E1F46B966FAD60
:103090006B976C967FAD6C976D968FAD6D976E96B6
:1030A0009FAD6E970E94EA02E0915103F0915203A6
:1030B0004189528963897489141615061606170604
:1030C000C4F2DACF235031092230310508F07FCE27
:1030D000A6966CAD7DAD8EAD9FADA6970E94EA021F
:1030E000882309F474CEE0915103F0915203118AC0
:1030F000128A138A148A68EC70E080E090E00E94E3
:10310000AB0280915303909154030E946703E091B6
:103110005303F09154038185928590935C038093CF
:103120005B0320915503309156032430310529F477
:1031300090936D0380936C03A3CF90936F03809360
:103140006E039ECF8430910511F1059709F0FCCEF6
:103150001092A6011092A50106C082E090E0909323
:10316000A6018093A5016091790370917A038FE4A1
:103170000BC081E090E09093A6018093A50160913F
:10318000790370917A0383E40E94AD06DDCE82E07C
:1031900090E09093A6018093A50180916C0390919B
:1031A0006D039C01215031092F36334010F08CEB18
:1031B00092E09093BC018093BB016091BB01709140
:1031C000BC0182E5E1CF81E090E09093A60180937D
:1031D000A50180916E0390916F039C0121503109EC
:1031E0002F36334010F08DE290E09093BA01809337
:1031F000B9016091B9017091BA018EE4C5CFE7E6DB
:10320000CE16E8E9DE06EAE9EE06E6EAFE0609F48D
:103210003CCC0CF059C02DEFC21622E0D2062AE9B0
:10322000E20626EAF20609F42BCB4DEDC41642E283
:10323000D4064AE9E40646EAF40611F00C94B00E0E
:103240008091A7019091A801019711F00C94B00E04
:103250008091B7019091B801892B11F00C94960ED2
:103260001091890111113ECB0E94DE02609385010D
:1032700070938601809387019093880111114FCB41
:103280004091B60164E670E081E090E00E9436046F
:1032900000918201109183010430110514F003E0C4
:1032A00010E00F5F1F4F10938301009382010430E1
:1032B000110509F083CB4091B60164E670E082E02D
:1032C00090E00E9436047ACB87E5C81688EAD806D3
:1032D0008AE9E80686EAF80609F437CB9DE3C916C1
:1032E00092ECD9069AE9E90696EAF90609F4CDCBFB
:1032F000ADE5CA16A2EADA06AAE9EA06A6EAFA06DD
:1033000009F49FCA0C94B00EB7E6CB16B8E9DB06F9
:10331000BAE9EB06B6EAFB0609F4B7CBB4F4FDEF65
:10332000CF16F2E0DF06FAE9EF06F6EAFF0609F447
:10333000A7CA2DEDC21622E2D2062AE9E20626EA43
:10334000F20609F47DCF0C94960E47E5C41648EAC0
:10335000D4064AE9E40646EAF40609F4F6CA8DE31F
:10336000C81682ECD8068AE9E80686EAF80609F467
:103370008CCB9DE5C91692EAD9069AE9E90696EA48
:10338000F90609F45ECA0C94960ECF93DF93C091B0
:103390003403D09135032097E1F0FE01329720816C
:1033A000318146E0429FC001439F900D1124C80F18
:1033B000D91F9E018091340390913503269782177F
:1033C000930721F0CE010E940C05F3CF02970E94D3
:1033D000F71C88E393E0DF91CF910C940C051F93C9
:1033E000FC0199278827BC01E89411911032E9F378
:1033F000193010F01E30C8F31B3251F01D3249F461
:10340000689406C00E94161A610F711D811D911DDE
:10341000119110531A30B0F33EF490958095709549
:1034200061957F4F8F4F9F4F1F910895592F482FC0
:10343000372F262F660F771F881F991F660F771F5C
:10344000881F991F620F731F841F951F660F771FB8
:10345000881F991F08950E946D1A08F481E008954D
:10346000E89409C097FB3EF490958095709561951E
:103470007F4F8F4F9F4F9923A9F0F92F96E9BB27D4
:103480009395F695879577956795B795F111F8CF50
:10349000FAF4BB0F11F460FF1BC06F5F7F4F8F4FBB
:1034A0009F4F16C0882311F096E911C0772321F0B1
:1034B0009EE8872F762F05C0662371F096E8862F49
:1034C00070E060E02AF09A95660F771F881FDAF7A0
:1034D000880F9695879597F90895990F0008550FCD
:1034E000AA0BE0E8FEEF16161706E807F907C0F08A
:1034F00012161306E407F50798F0621B730B840B92
:10350000950B39F40A2661F0232B242B252B21F46B
:1035100008950A2609F4A140A6958FEF811D811D0B
:1035200008950E94A41A0C94151B0E94071B38F0E2
:103530000E940E1B20F0952311F00C94FE1A0C949F
:10354000041B11240C94491B0E94261B70F3959FA9
:10355000C1F3950F50E0551F629FF001729FBB278A
:10356000F00DB11D639FAA27F00DB11DAA1F649F26
:103570006627B00DA11D661F829F2227B00DA11DD9
:10358000621F739FB00DA11D621F839FA00D611D5F
:10359000221F749F3327A00D611D231F849F600D80
:1035A000211D822F762F6A2F11249F5750409AF0A9
:1035B000F1F088234AF0EE0FFF1FBB1F661F771F35
:1035C000881F91505040A9F79E3F510580F00C9400
:1035D000FE1A0C94491B5F3FE4F3983ED4F38695A2
:1035E00077956795B795F795E7959F5FC1F7FE2BA0
:1035F000880F911D9695879597F9089597F99F677C
:1036000080E870E060E008959FEF80EC089500246A
:103610000A941616170618060906089500240A9437
:1036200012161306140605060895092E0394000CBD
:1036300011F4882352F0BB0F40F4BF2B11F460FF4C
:1036400004C06F5F7F4F8F4F9F4F089557FD905875
:10365000440F551F59F05F3F71F04795880F97FB56
:10366000991F61F09F3F79F0879508951216130610
:103670001406551FF2CF4695F1DF08C0161617063F
:103680001806991FF1CF8695710561050894089574
:10369000E894BB2766277727CB0197F90895F99916
:1036A000FECF92BD81BDF89A992780B50895262F47
:1036B000F999FECF1FBA92BD81BD20BD0FB6F89417
:1036C000FA9AF99A0FBE019608950E94A71BA59F2A
:1036D000900DB49F900DA49F800D911D112408950D
:1036E0002F923F924F925F926F927F928F929F9212
:1036F000AF92BF92CF92DF92EF92FF920F931F9300
:10370000CF93DF93CDB7DEB7CA1BDB0B0FB6F894B0
:10371000DEBF0FBECDBF09942A88398848885F84F0
:103720006E847D848C849B84AA84B984C884DF8061
:10373000EE80FD800C811B81AA81B981CE0FD11D45
:103740000FB6F894DEBF0FBECDBFED010895A29F66
:10375000B001B39FC001A39F700D811D1124911D65
:10376000B29F700D811D1124911D08950E94BD1BF3
:103770006894B1110C94491B08950E942E1B88F087
:103780009F5798F0B92F9927B751B0F0E1F0660F25
:10379000771F881F991F1AF0BA95C9F714C0B13066
:1037A00091F00E94481BB1E008950C94481B672FCC
:1037B000782F8827B85F39F0B93FCCF38695779595
:1037C0006795B395D9F73EF490958095709561957E
:1037D0007F4F8F4F9F4F0895DB018F939F930E94E0
:1037E000651BBF91AF91A29F800D911DA39F900D6E
:1037F000B29F900D1124089597FB072E16F40094A4
:1038000007D077FD09D00E94471C07FC05D03EF485
:10381000909581959F4F0895709561957F4F08957C
:10382000A1E21A2EAA1BBB1BFD010DC0AA1FBB1FC4
:10383000EE1FFF1FA217B307E407F50720F0A21B36
:10384000B30BE40BF50B661F771F881F991F1A94A3
:1038500069F760957095809590959B01AC01BD01CD
:10386000CF010895EE0FFF1F0590F491E02D09940C
:103870000E94A71BB7FF0895821B930B0895B7FF03
:103880000C94651B0E94651B821B930B0895AA1B59
:10389000BB1B51E107C0AA1FBB1FA617B70710F03B
:1038A000A61BB70B881F991F5A95A9F7809590956D
:1038B000BC01CD0108950F931F93CF93DF93823006
:1038C000910510F482E090E0E0919603F091970367
:1038D00030E020E0B0E0A0E0309799F42115310508
:1038E00009F44AC0281B390B24303105D8F58A81E8
:1038F0009B816115710589F1FB0193838283FE0130
:1039000011C0408151810281138148175907E0F0AD
:103910004817590799F4109761F012960C93129773
:1039200013961C933296CF01DF91CF911F910F9187
:1039300008950093960310939703F4CF2115310552
:1039400051F04217530738F0A901DB019A01BD017C
:10395000DF01F801C1CFEF01F9CF90939703809376
:103960009603CDCFFE01E20FF31F81939193225076
:10397000310939832883D7CF20919403309195035F
:10398000232B41F4209104013091050130939503DC
:1039900020939403209102013091030121153105F8
:1039A00041F42DB73EB74091060150910701241B09
:1039B000350BE0919403F0919503E217F307A0F41F
:1039C0002E1B3F0B2817390778F0AC014E5F5F4F75
:1039D0002417350748F04E0F5F1F5093950340930F
:1039E0009403819391939FCFF0E0E0E09CCFCF933D
:1039F000DF930097E9F0FC01329713821282A091C5
:103A00009603B0919703ED0130E020E01097A1F408
:103A100020813181820F931F20919403309195036F
:103A20002817390709F061C0F0939503E0939403D8
:103A3000DF91CF910895EA01CE17DF07E8F54A81BB
:103A40005B819E0141155105B1F7E901FB83EA83D2
:103A500049915991C40FD51FEC17FD0761F480817E
:103A600091810296840F951FE90199838883828151
:103A700093819B838A83F0E0E0E012968D919C9184
:103A800013970097B9F52D913C911197CD010296AE
:103A9000820F931F209194033091950328173907C3
:103AA00039F6309751F51092970310929603B09320
:103AB0009503A0939403BCCFD383C28340815181EB
:103AC000840F951FC817D90761F44E5F5F4F888137
:103AD0009981480F591F518340838A819B81938329
:103AE00082832115310509F0B0CFF0939703E0935D
:103AF00096039ECFFD01DC01C0CF13821282D7CF87
:103B0000B0E0A0E0E6E8FDE10C94721B8C010097A8
:103B100051F4CB010E945B1C8C01C801CDB7DEB70C
:103B2000E0E10C948E1BFC01E60FF71F9C01225074
:103B30003109E217F30708F49DC0D901CD91DC915A
:103B40001197C617D70798F0C530D10530F3CE01CD
:103B500004978617970708F3C61BD70B2297C193C4
:103B6000D1936D937C93CF010E94F71CD6CF5B015C
:103B7000AC1ABD0A4C018C0E9D1EA0919603B0910B
:103B80009703512C412CF12CE12C109731F58091A9
:103B90009403909195038815990509F05CC0461629
:103BA000570608F058C080910201909103010097D8
:103BB00041F48DB79EB74091060150910701841BD7
:103BC000950BE817F90708F055C0F0939503E093BB
:103BD0009403F90171836083A0CF8D919C9111971B
:103BE00012966C90129713967C901397A815B905AE
:103BF00059F56C0142E0C40ED11CCA14DB0420F15B
:103C0000AC014A195B09DA011296159780F06282BD
:103C1000738251834083D9016D937C93E114F10445
:103C200071F0D7011396FC93EE93129776CF2296FC
:103C30008C0F9D1FF90191838083F301EFCFF093E7
:103C40009703E093960369CF4816590608F42C01B0
:103C50007D01D3019ACFCB010E945B1C7C010097B0
:103C600049F0AE01B8010E943D1EC8010E94F71C38
:103C7000870153CF10E000E050CFFB01DC0102C010
:103C800001900D9241505040D8F70895FB01DC019E
:103C900001900D920020E1F70895AEE0B0E0E3E579
:103CA000FEE10C947E1B0D891E898F89988D26E07C
:103CB0002C831A83098397FF02C080E090E8019764
:103CC0009E838D83AE01455E5F4F698D7A8DCE01F7
:103CD00001960E94A01E4D815E8157FD0AC02F8172
:103CE0003885421753070CF49A01020F131FF8018D
:103CF00010822E96E4E00C949A1BAEE0B0E0E3E86C
:103D0000FEE10C947E1B0D891E8986E08C831A834C
:103D100009838FEF9FE79E838D83AE01475E5F4FE0
:103D20006F89788DCE0101960E94A01E2F81388563
:103D3000020F131FF80110822E96E4E00C949A1BD8
:103D4000ABE0B0E0E6EAFEE10C94701B7C013B01C5
:103D50008A01FC0117821682838181FFC8C1CE01CE
:103D600001965C01F7019381F30193FD859193FF27
:103D700081913F01882309F453C1853239F493FDC1
:103D8000859193FF81913F01853229F4B70190E03D
:103D90000E949020E7CF912C212C312CFFE1F315CC
:103DA00038F08B3211F190F4803209F1833229F12D
:103DB00037FC3CC020ED280F2A3050F536FE20C0DD
:103DC0008AE0989E200D1124922E06C08D3291F02B
:103DD000803371F7689430F8F30193FD859193FF78
:103DE00081913F018111DACF21C0689431F8689444
:103DF00032F8F2CF689433F8EFCF689434F8ECCF10
:103E0000EAE02E9E200D1124222E689435F8E4CF8E
:103E10008E3229F436FC04C1689436F8DDCF8C3636
:103E200019F4689437F8D8CF8836B1F2982F9F7D6F
:103E300095549330E0F08336A1F18337C1F1833597
:103E400009F063C02801F2E04F0E511CF801C08058
:103E5000D180692D70E036FC02C06FEF7FEFC601A4
:103E60000E947A204C01689437F882010AC00C5FE6
:103E70001F4FFFE3F98388248394912C6501E89414
:103E800037F833FE2DC0522C8114910471F5552062
:103E900009F468CFB70180E290E00E9490205A9424
:103EA000F6CFF801808189830E5F1F4FE4CF280190
:103EB000F2E04F0E511CF801C080D180692D70E0F6
:103EC00036FC02C06FEF7FEFC6010E9485204C01D7
:103ED0008201D5CFB70180E290E00E9490202A9421
:103EE0002814190409F0B0F7CECFF60137FC8591FC
:103EF00037FE81916F01B70190E00E949020511030
:103F00005A94F1E08F1A9108BFCF843619F08936A0
:103F100009F077C0F80137FE6BC060817181828142
:103F200093810C5F1F4FF32DFF763F2E97FF09C043
:103F300090958095709561957F4F8F4F9F4F6894B6
:103F400037F82AE030E0A5010E94C020C82ECA1828
:103F50008C2C432C36FE0CC0E89440F8C91440F475
:103F600034FE05C032FC03C0F32DFE7E4F2E892C9B
:103F700044FE95C0FE01EC0DF11D8081803309F0F7
:103F800087C0242D297E422E842D8870582E43FC14
:103F900095C040FE8FC09C2C821418F42C0C922CDF
:103FA000981844FE91C0B70180E390E00E949020F1
:103FB00042FE09C088E790E041FE02C088E590E03B
:103FC000B7010E949020C91408F48AC0CA94D12C69
:103FD0009FEFC91AD90ACA0CDB1CF60182916F0146
:103FE000B70190E00E949020AC14BD04B1F74FCF10
:103FF00060817181072E000C880B990B0E5F1F4F9B
:1040000092CFD32CE894D4F82AE030E0853739F108
:10401000232D297FD22E8F3601F148F48835A9F05F
:10402000F701868197812B96E2E10C948C1B8037F7
:1040300049F08837A9F7D4FE02C06894D2F820E18D
:1040400030E00DC06894D4F8F6CF34FE03C0822F60
:104050008660D82E20E132E002C028E030E0F8018E
:10406000D7FE0FC060817181828193810C5F1F4FE9
:10407000A5010E94C020C82ECA183D2CE89437F82C
:1040800067CF6081718190E080E00E5F1F4FF0CFBD
:1040900042FC02C0839478CF8394839475CF842D9F
:1040A000867809F471CFF6CFB70180E290E00E94E4
:1040B000902083948214C0F3512C73CF522C581843
:1040C000821408F46ECFF8CF842D867809F47BCF64
:1040D0008BE241FE80E247FC8DE2B70190E071CFB8
:1040E000B70180E390E00E9490209A946CCF8FEF0C
:1040F0009FEF99CFFC010590615070400110D8F7F7
:10410000809590958E0F9F1F0895FC01615070401F
:1041100001900110D8F7809590958E0F9F1F0895FC
:104120000F931F93CF93DF93182F092FEB018B81F0
:1041300081FD09C01FEF0FEF812F902FDF91CF91ED
:104140001F910F91089582FF14C02E813F818C81B1
:104150009D81281739073CF4E881F981CF01019648
:104160009983888310838E819F8101969F838E839C
:10417000E3CFE885F985812F0995892BA1F3DACF63
:10418000FA01AA27283051F1203181F1E8946F9388
:104190006E7F6E5F7F4F8F4F9F4FAF4FB1E03ED02E
:1041A000B4E03CD0670F781F891F9A1FA11D680FCC
:1041B000791F8A1F911DA11D6A0F711D811D911DFF
:1041C000A11D20D009F468943F912AE0269F112474
:1041D0003019305D3193DEF6CF010895462F4770D8
:1041E000405D4193B3E00FD0C9F7F6CF462F4F7033
:1041F000405D4A3318F0495D31FD4052419302D091
:10420000A9F7EACFB4E0A695979587957795679536
:10421000BA95C9F700976105710508959B01AC0136
:104220000A2E06945795479537952795BA95C9F75D
:10423000620F731F841F951FA01D089510E0C2E632
:10424000D0E004C0FE010E94321C2196C336D10783
:06425000C9F7F894FFCF4E
:1042560090010000980380003130370047656D6992
:104266006E69466C617450616E656C50726F0005C4
:1042760002C2010603BC02010001000001010000A8
:10428600010001010000010000000024018E00BBB6
:10429600007101EC00CA00DE002A25632573256340
:1042A600002A2563256425630025640025644D25C1
:1042B600644C25644325644425644325644F00000B
:00000001FF
